:0800000011308A0017290000ED
:10002000FF00030E8301A1000A08A0008A01040852
:10003000A2007708A3007808A4007908A5007A0830
:10004000A600831383128C308400001C29280C180E
:100050003E288B1E2D280B194128220884002308D6
:10006000F7002408F8002508F9002608FA002008FF
:100070008A00210E8300FF0E7F0E09008A110A12EA
:100080002F298A110A12A3298E30F70003171A08A4
:10009000F8001908F900FA01F808031D5928790831
:1000A000F800F9010830F702F808031D5928F70194
:1000B00061280310F81B6028F90DF80DF703592883
:1000C000F813031308000317190803192929A500B9
:1000D0001D0803192929A502031C73287F30A507D1
:1000E0000318292979288130A502031C292903191D
:1000F00029292508F700F801F901FA01A4011A08D5
:10010000A300A3171B08A2001C08A1001930A5001A
:100110002008A10203189C280130A20203189C2881
:10012000A30203189C28A40203189C28A40AA30A6B
:10013000A20A2008A107CE281F08A2020318B72888
:100140000130A3020318B728A4020318B728A40A91
:10015000A30A1F08A2072008A107031CCE28A20A91
:10016000031DCE28A30A031DCE28A40ACE281E08EC
:100170008038A3020318CD280130A4020318CD282B
:10018000A40A1E088038A3071F08A207031CAB2877
:10019000A30A031DAB28A40AAB287A14A50BD12807
:1001A000DC280310A10DA20DA30DA40D0310FA0D60
:1001B000F90DF80DA60D8828261CE4280310F80C6C
:1001C000F90CFA0CA60CE728F70303192929A61B3A
:1001D00010290310A10DA20DA30DA40D2008A1024A
:1001E0000318FC280130A2020318FC28A3020318FC
:1001F000FC28A402031C1F291F08A20203180729B8
:100200000130A30203180729A402031C1F291E089A
:100210008038A302031810290130A402031C1F29EF
:10022000FA0A031D1F29F90A031D1F29F80A031DD5
:100230001F29F70A03192929F80CF90CFA0C1A08D6
:10024000A5001E08A506A51F2729F8172D29F813B4
:100250002D29F701F801F901FA01031308004108FB
:100260000317980003134008031797009A01FF3003
:10027000990010309B00F701FA01980C970C031CB1
:1002800047291908F7070318FA0A1A08FA07FA0C97
:10029000F70CF90CF80C9B0B3D29790898007808AD
:1002A000970003130108031797070318980A180803
:1002B0009A0017089900031344207A0803179C003A
:1002C00079089B0078089A00770899008030A00090
:1002D0009F019E017E309D00031363207A08C500B4
:1002E0007908C4007808C3007708C20045080317DE
:1002F0009C000313440803179B00031343080317D0
:100300009A000313420803179900A0019F012830A7
:100310009E0082309D00031363207A08C50079088F
:10032000C4007808C3007708C200C101C001810180
:100330008F018E01831609100130831289060C107B
:100340008A110A122D28C00A0319C10A0B118A1139
:100350000A122D280D050D052310C12B5318B120AD
:10036000A0127310A82129103218B119A03BF73B35
:10037000AE36EC306217633DA0060A0083165308C0
:10038000D5005208D4005508FA005408840083139D
:100390007A18831780080319D129D40A0319D50ABA
:1003A000C32952085402F7005508FA005308031CE9
:1003B000530FFA027708F800831208008316031718
:1003C0008C170C14000000000318152A83120C0867
:1003D0007F3983160313D300831203170D08831686
:1003E0000313D400831203170F0883160313D500D9
:1003F000530883120C1EFA2999008316540883129D
:1004000003178D00831603135508831203178F00FB
:1004100083168C170C14000000000313D20B112A52
:10042000132A0317152A402A031783120C0D0E0DE9
:100430007F3983160313D300831203170D08831625
:100440000313D400831203170F0883160313D50078
:10045000530883120C1E2A2A99008316540883120B
:1004600003178D00831603135508831203178F009B
:100470008D0A03198F0A031083160313D20BDF2989
:1004800083120800800803195F2A8316D301040829
:10049000D2005310831B5314000883120C1E4E2AE3
:1004A0009900831652088400831353188317840A13
:1004B000031D5D2A8312850A83168312422A0800CF
:1004C00024308316A0004930A1006430A2003A30E5
:1004D000A3002030A4006D30A5006130A600693073
:1004E000A7006E30A8002E30A9006330AA0020308B
:1004F000AB003230AC003930AD003030AE003730B8
:10050000AF002030B0003230B1003030B2003130B6
:10051000B3003330B4002D30B5003030B600343085
:10052000B7002D30B8003130B9003330BA00203078
:10053000BB003230BC003030BD003A30BE00353038
:10054000BF003230C0003A30C1003230C200353016
:10055000C3005A30C4002030C5006B30C600613083
:10056000C7006B30C8006C30C9006930CA006B30FE
:10057000CB002030CC002430CD00CE01D301A03000
:10058000D2008312BE2101307802A03E8400831382
:100590000008243C031DD82A8316D301A030D200C2
:1005A0008312BE2101307802A03E840083138001B3
:1005B000AA3003178D0001308F0003100D30831611
:1005C0000313D2008312DE212B30840083134222D6
:1005D000B13003178D0001308F00031418308316DB
:1005E0000313D2008312DE2123300C1EF52A99005A
:1005F000A4308400831342220D300C1EFD2A990082
:100600000A300C1E012B99008A110A16BB29831689
:1006100008148810831288100D2B0E2B8316881057
:1006200083128814132B142B8316081083120810BE
:10063000192B1A2B83168810831288100330F700A9
:10064000F70B202B8316881083128814272B282B56
:10065000831608142B2B2C2B88108312881008006B
:10066000AF308400831300080319432B0230F800D5
:10067000F701F70B392BF80B382B9730F700F70BF6
:100680003F2B800B362B080083160814881083122A
:1006900088100330F700F70B4B2BF1017108083C71
:1006A000031C642B83168810831288140330F70010
:1006B000F70B582B83168810831288100330F7002D
:1006C000F70B602BF10A4E2B072314308316AF0073
:1006D000831230238A110A16C5298030831C732B9C
:1006E0008316C50683128316CA01CB014108C900CF
:1006F0004508C90640080319612CC800F7004408E2
:1007000003196A2CC8020319062C031CC42B4508C4
:10071000CE00CE174608CD004708CC00CB01031011
:10072000CE0CCD0CCC0CCB0CC80B8E2BC91F9B2B2D
:100730004A147E2C4A1048104A16C3308400831392
:10074000932C4A12C91BAE2B481CB92BCE0CCD0CD6
:10075000CC0CCB0CF70A0319792CB92BCE1BBC2B74
:100760000310CB0DCC0DCD0DCE0DF7030319792C55
:10077000AE2B4A17262C4A134108C900C91FC22BA9
:10078000CE17722CCE13722C4408C800F700400814
:10079000C8024108CE00CE174208CD004308CC0065
:1007A000CB010310CE0CCD0CCC0CCB0CC80BD02B3A
:1007B000C91FDD2BCA147E2CCA104810CA16C730B8
:1007C00084008313932CCA12C91BF02B481CFB2BEB
:1007D000CE0CCD0CCC0CCB0CF70A0319792CFB2BCF
:1007E000CE1BFE2B0310CB0DCC0DCD0DCE0DF70384
:1007F0000319792CF02BCA17262CCA134508C900F7
:10080000C91F042CCE17722CCE13722C4508CE00B3
:10081000CE174608CD004708CC00C91F132CCE13B5
:100820004A157E2C4A11CB014810C3308400831333
:10083000932CC91B3C2C4108C900481C262CCE0C0B
:10084000CD0CCC0CCB0CF70A0319792CCB1F372C11
:10085000CC0A031D372CCD0A031D372CCE0A031DED
:10086000372CCE0CCD0CCC0CF70A0319792C4A1B73
:10087000BB2BCA1BFD2B5B2C8030CE06CE1F442C1D
:100880007E2C4508C900512C4108C900CE08031D23
:10089000512CCD08031D512CCC08031D512CF70100
:1008A000722CCE1B5B2C0310CB0DCC0DCD0DCE0DC1
:1008B000F70B512C792CC91F5F2CCE17722CCE133D
:1008C000722C4408F7004508CE004608CD004708C2
:1008D000CC00722C4008F7004108CE004208CD0041
:1008E0004308CC004E08F8004D08F9004C08FA0007
:1008F000B12CF701F801F901FA01B12CCB01CC09B7
:10090000CD09CE09CB09CB0A031D8C2CCC0A031DC3
:100910008C2CCD0A0319CE0A4A189A2BCA18DC2B44
:100920004A19122C412C0008CC07031C9D2CCD0A1F
:10093000031D9D2CCE0A0319481484030008CD071B
:10094000031CA52CCE0A0319481484030008801F39
:10095000803ACE07031848144A1AA12BCA1AE32B6F
:10096000192C831208002F112F0883168700831279
:1009700007111308883093008316140C031CBD2C38
:100980008312130893018316140C031CC42C8312C6
:100990001308F10013088A3093008316140C031C0B
:1009A000CE2C8312130893018316140C031CD52C30
:1009B00083121308F20013088C3093008316140C72
:1009C000031CDF2C8312130893018316140C031CE1
:1009D000E62C83121308F30013088E30930083165D
:1009E000140C031CF02C8312130893018316140CAF
:1009F000031CF72C83121308F400130890309300A3
:100A00008316140C031C012D831213089301831603
:100A1000140C031C082D83121308F50013089230E0
:100A200093008316140C031C122D831213089301D8
:100A30008316140C031C192D83121308F6001308D7
:100A4000943093008316140C031C232D8312130877
:100A500093018316140C031C2A2D83121308FB0028
:100A60001308963093008316140C031C342D831244
:100A7000130893018316140C031C3B2D83121308D7
:100A8000FC00130893018316140C031C442D8312DD
:100A90002F112F0883168700831207158316A101D3
:100AA0007108A000A00DA10DA00DA10DA00DA10D1C
:100AB000A00DA10DA00DA10DE030A005720CF70056
:100AC000F70CF70C1F30F7057708A0070318A10AE9
:100AD000720807398312A7018B1BA7178B13031703
:100AE0009A01990003134420A71B8B17A7018B1BA6
:100AF000A7178B137A0803179C0079089B007808C6
:100B00009A0077089900A0019F019E0182309D0004
:100B100003136320A71B8B1777088316A40078089C
:100B2000A5007908A6007A08A7008312A7018B1BED
:100B3000A7178B1383162108831203179A008316B5
:100B40000313200883120317990003134420A71BE3
:100B50008B1783107A088316C3007908C2007808BF
:100B6000C1007708C0002708C7002608C60025086E
:100B7000C5002408C40083126D237A08B3007908E5
:100B8000B2007808B1007708B00073081F39FA0185
:100B90008316A100A0017408A0070318A10A8312FC
:100BA000A7018B1BA7178B1383162108831203172A
:100BB0009A00831603132008831203179900031366
:100BC0004420A71B8B17A7018B1BA7178B137A0831
:100BD00003179C0079089B0078089A007708990011
:100BE000A0019F019E018C309D0003136320A71B71
:100BF0008B1777088316A0007808A1007908A20057
:100C00007A08A30083142308C3002208C200210825
:100C1000C1002008C000C701C6014030C5008030B7
:100C2000C40083126D237A08B7007908B6007808EB
:100C3000B5007708B400803075028316A101A000CA
:100C4000A100A0017608A0070318A10A8312A7013A
:100C50008B1BA7178B1383162108831203179A0087
:100C600083160313200883120317990003134420EB
:100C7000A71B8B17A7018B1BA7178B137A080317CA
:100C80009C0079089B0078089A0077089900A001D9
:100C90009F019E018D309D0003136320A71B8B17BE
:100CA00077088316A0007808A1007908A2007A08C6
:100CB000A30083142308C3002208C2002108C10036
:100CC0002008C000C701C601C5018030C4008312DE
:100CD0006D237A08BB007908BA007808B900770854
:100CE000B800FA017B088316A100A0017C08A007C8
:100CF0000318A10A8312A7018B1BA7178B13831656
:100D00002108831203179A00831603132008831205
:100D10000317990003134420A71B8B17A7018B1BF4
:100D2000A7178B137A0803179C0079089B00780893
:100D30009A0077089900A0019F019E0197309D00BD
:100D400003136320A71B8B177A08BF007908BE0026
:100D50007808BD007708BC0071087204730474043D
:100D6000750476047B047C04FF3C031DBB2E01301C
:100D7000F800BE2EBE2E0030F800BE2E8A110A16D4
:100D8000C8290830F80000008711AF112F0883161A
:100D900087000000FB0D83120712031CD52E2F16AF
:100DA0002F0883168700D92E83122F122F0883163F
:100DB000870000008312AF152F0883168700831267
:100DC000871DE02EF80BC32E00008711AF112F08EE
:100DD00083168700000083122F162F0883168700C2
:100DE000000000008312AF152F08831687008312BE
:100DF000871DF82EF8010000071A78148711AF112B
:100E00002F0883168700831207122F122F088316CC
:100E10008700831208002F162F0883168700000012
:100E20008312AF152F088316870000008312071264
:100E30002F122F0883168700000083128711AF112D
:100E40002F08831687008030FB008312C126FE30F6
:100E5000FB00C1262F122F08831687000000831283
:100E6000AF152F08831687008312871D352F0000CA
:100E7000392F00002F162F088316870000008312D9
:100E80008A110A16CE2908308316B002031C542F8B
:100E9000B030840083130310800C00080319542F12
:100EA000522F0000800B512F8312080083168610EA
:100EB0008312861002308316AF00F830B000831220
:100EC00043278316AF0B5D2F86140230AF00F83036
:100ED000B000831243278316AF0B672F861483124B
:100EE00008008316B0013008073C031C932F8610BE
:100EF000831286107B2F7C2F03148316AF0C0318EC
:100F0000852F83128610872F8316831286148316EB
:100F100086102730F700F70B8B2F8E2F8614902F1B
:100F2000912FB00A732F831208008316B101310884
:100F3000073C031CB62F8610831286109F2FA02F0C
:100F4000831686140530F700F70BA42F861483123E
:100F50008618AC2F0310AD2F03148316B20C4F303C
:100F6000F700F70BB12FB42FB10A972F3208F80012
:100F70008312080080308316AD000330F700F70BB2
:100F8000BF2FAC012C08073C031CE02F88108312F4
:100F9000881083162B082D050319D02F0814D42F81
:100FA0000810831208108316D52FD62F88108312AD
:100FB0008814DA2FDB2F03108316AD0CAC0AC22F76
:100FC000881083128810E42FE52F831608142E1042
:100FD0008312081CEE2F83162E148312831688109A
:100FE00083128814F32FF42F83168810831288102D
:0E0FF000003083162E180130F800831208001E
:101000008316440803197128CC0048080319712875
:10101000CC07031812287F30CC02031C7128031957
:10102000712816288130CC07031871284C08F70066
:10103000F801F901FA014508D000D0174608CF00A1
:101040004708CE001830CC00CD014E1C3F284B087D
:10105000FA07031C3128F90A031D3128F80A03197D
:10106000CD174A08F907031C3828F80A0319CD17C9
:101070004908C600C6174608F8070318CD17CD0D56
:10108000F80CF90CFA0CD00CCF0CCE0C0310CC0BD6
:1010900024280130F70703187128F81B5628D00DB3
:1010A000FA0DF90DF80DF70303197128D01F672801
:1010B000FA0A031D6728F90A031D6728F80A031DA9
:1010C0006728F80CF90CFA0CF70A0319712845087F
:1010D000CD004908CD06CD1F6F28F8177528F813E5
:1010E0007528F701F801F901FA018312080071105F
:1010F0008A1156278A15CC308316AF008A118312C5
:1011000071278A1544308316AF008A118312712724
:101110008A15F2017208C73C031C9F288A11952783
:101120008A1571107818711471189F280130831670
:10113000AF008A11831230238A15F20A8A288A1195
:1011400056278A15CC308316AF008A118312712777
:101150008A15BE308316AF008A11831271278A1553
:10116000F2017208083C031CCB28A0307207F8007B
:10117000FA010318FA0A7808FB007A08FC008A11C1
:1011800095278A157B08840083137C1883177808B9
:101190008000F20AB12883162708103C031D3B2962
:1011A0002108FA0020088312A7018B1BA7178B13B5
:1011B000031799007A089A008A11031344208A15AC
:1011C000A71B8B177A08F6007908F5007808F40059
:1011D0007708F30076088316C7007508C600740800
:1011E000C5007308C400CB01CA014030C90081307A
:1011F000C800831200207708FB007808FC007908FB
:10120000FD007A08FE00A7018B1BA7178B13760839
:1012100003179C0075089B0074089A0073089900D6
:10122000A0019F019E0181309D008A11031363205C
:101230008A15A71B8B1783107E088316C3007D08B1
:10124000C2007C08C1007B08C0007A08C70079088A
:10125000C6007808C5007708C4008A1183126D2380
:101260008A157A08F6007908F5007808F4007708FE
:10127000F30043298316F6016630F500D530F400FB
:101280008D30F30083127308F7007408F8007508B6
:10129000F9007608FA008A110A16EF298316081455
:1012A000881083128810542955298316AC01AB018C
:1012B0002C08013C031C7529031D62292B085D3C89
:1012C000031C7529081483120818692983167529C7
:1012D000831201308316AF008A11831230238A15DE
:1012E0008316AB0A0319AC0A582983120800831627
:1012F000AD01AC01AB012B08073C031C992903107D
:10130000AC0DAD0D881083128814862987298316A9
:1013100008148312081C902983162C148F29831219
:101320008316881083128810952996298316AB0A94
:101330007B290810831208109D299E298316881086
:10134000831288140330F700F70BA4298316881042
:1013500083128810AB29AC2983160814AB012B0823
:10136000073C031CCD290310AC0DAD0D8810831272
:101370008814BA29BB29831608148312081CC429AF
:1013800083162C14C32983128316881083128810A5
:10139000C929CA298316AB0AAF290814CF29D02935
:1013A0008810831288140330F700F70BD5298316B1
:1013B00088108312881083162C08F8002D08F90075
:1013C0008312080083163D08C4004108C406C41FE8
:1013D000EE2903110310BD1B0314212A3D08C4008C
:1013E0004008C5003C08C5020319FC29C41F212A76
:1013F0000308013A8300212A4108C5003D08C502BF
:101400000319082AC41F212A0308013A8300212A4C
:101410004208C5003E08C5020319142AC41F212A28
:101420000308013A8300212A4308C5003F08C5028A
:101430000319202AC41F212A0308013A8300212A04
:101440000310831208000830FC007708FD002F16F7
:101450002F088316870000008312AF152F0883160C
:1014600087008312871D322A071A0314071E0310F0
:10147000F80D0000AF112F08831687008312871123
:10148000FC0B272A2F162F088316870000008312D3
:1014900007127D080319512A2F122F08831687007F
:1014A00083120000AF152F08831687008312871D53
:1014B000572A00008711AF112F08831687000000FC
:1014C000831207122F122F08831687008312080039
:1014D0002F162F088316870000008312AF152F08E0
:1014E0008316870000008312871D742A07122F12AB
:1014F0002F0883168700000083128711AF112F0871
:10150000831687008030FB008A118312C1268A155A
:10151000E330FB008A11C1268A152F122F0883168B
:10152000870000008312AF152F08831687008312EF
:10153000871D982A00009C2A00002F162F0883166A
:10154000870000006430AF008A11831230238A15AF
:101550002F162F088316870000008312AF152F085F
:10156000831687000000831207122F122F0883169C
:101570008700000083128711AF112F0883168700A0
:101580008130FB008A118312C1268A150130F700D1
:1015900023227808F1000130F70023227808F200B6
:1015A000F70123227808F3002F122F0883168700F3
:1015B00000008312AF152F08831687008312871D42
:1015C000DF2A0000E32A00002F162F088316870069
:1015D0000000F20CF20C3F30F205FC017108FB0038
:1015E000FC00FB01720EF700F030F70577087B076F
:1015F000F4007C08F5000318F50A8312A7018B1B81
:10160000A7178B13750803179A00740899008A119D
:10161000031344208A15A71B8B177708FB00780853
:10162000FC007908FD007A08FE00A7018B1BA717B4
:101630008B137A0803179C0079089B0078089A009E
:1016400077089900A001FF309F007F309E008E3008
:101650009D008A11031363208A15A71B8B17523034
:101660008316C700B830C6002F30C5008630C400CE
:101670007A08CB007908CA007808C9007708C80042
:1016800083120020831066308316C300C200BB3073
:10169000C1008430C0007A08C7007908C600780805
:1016A000C5007708C4008A1183126D238A158A1138
:1016B0000A16982C2F162F08831687000000831215
:1016C000AF152F08831687000000831207122F1210
:1016D0002F0883168700000083128711AF112F088F
:1016E000831687008030FB008A118312C1268A1579
:1016F000E530FB008A11C1268A1564308316AF00DD
:101700008A11831230238A152F162F08831687001B
:1017100000008312AF152F08831687000000831284
:10172000871D902B07122F122F08831687000000A9
:1017300083128711AF112F08831687008130FB00B9
:101740008A118312C1268A150130F70023227808F6
:10175000F1000130F70023227808F200F70123227C
:101760007808F3002F122F088316870000008312D9
:10177000AF152F08831687008312871DBD2B00002D
:10178000C12B00002F162F08831687000000F20CD3
:10179000F20C3F30F205FC017108FB00FC00FB017C
:1017A000720EF700F030F70577087B07F4007C082D
:1017B000F5000318F50A8312A7018B1BA7178B13DB
:1017C000750803179A00740899008A1103134420BE
:1017D0008A15A71B8B177708FB007808FC0079088F
:1017E000FD007A08FE00A7018B1BA7178B137A0850
:1017F00003179C0079089B0078089A0077089900E5
:10180000A001FF309F007F309E008E309D008A1126
:10181000031363208A15A71B8B178316C701C60104
:101820007A30C5008530C4007A08CB007908CA0038
:101830007808C9007708C800831200208310831637
:10184000C301C201C030C1008130C0007A08C700A6
:101850007908C6007808C5007708C4008A11831289
:101860006D238A158A110A16A52C2F112F088316AD
:101870008700831207111308223093008316140C7B
:10188000031C3F2C8312130893018316140C031CB2
:10189000462C83122F112F088316870083120715F9
:1018A0000A308316AF008A11831230238A152F1154
:1018B0002F088316870083120711130884309300C2
:1018C0008316140C031C612C8312130893018316D6
:1018D000140C031C682C83121308F20013088630C2
:1018E00093008316140C031C722C831213089301AB
:1018F0008316140C031C792C83121308F1001308AF
:1019000093018316140C031C822C83122F112F08B1
:101910008316870083120715FC017208FB00FC0088
:10192000FB017108FB070318FC0A7C0CF4007B0C1C
:10193000F300F40CF30CF40CF30CF40CF30CF40CB7
:10194000F30CF40CF30C0330F405A7018B1BA71761
:101950008B13740803179A00730899008A110313F4
:1019600044208A15A71B8B177708FB007808FC001A
:101970007908FD007A08FE0083147A088316C300F4
:101980007908C2007808C1007708C000C701C60105
:101990007930C5008730C4008A1183126D238A15FF
:1019A0007708FB007808FC007908FD007A08FE0043
:1019B000A7018B1BA7178B137A0803179C007908C4
:1019C0009B0078089A00770899003330A0009F00A8
:1019D000AB309E0081309D008A11031363208A156D
:1019E000A71B8B177708FB007808FC007908FD001F
:1019F0007A08FE0083107A088316C3007908C200B3
:101A00007808C1007708C000C701C6015830C5007A
:101A10008330C4008A1183126D238A158A110A1635
:101A2000B42C2F112F088316870083120711130877
:101A3000243093008316140C031C1B2D83121308EF
:101A400093018316140C031C222D83122F112F08CF
:101A500083168700831207150A308316AF008A1198
:101A6000831230238A152F112F08831687008312C3
:101A700007111308803093008316140C031C3D2DAE
:101A80008312130893018316140C031C442D831234
:101A90001308F2001308823093008316140C031C01
:101AA0004E2D8312130893018316140C031C552D1D
:101AB00083121308F1002F112F0883168700831259
:101AC00007158316A1017208A000A100A0017108EA
:101AD000A0070318A10A210CF400200CF300F40C59
:101AE000F30CF40CF30CF40CF30CF40CF30CF40CFA
:101AF000F30C0330F40583122F112F08831687008F
:101B0000831207111308843093008316140C031CEE
:101B1000862D8312130893018316140C031C8D2D3C
:101B200083121308F2001308863093008316140CF6
:101B3000031C972D8312130893018316140C031CA6
:101B40009E2D83121308F100130893018316140CC1
:101B5000031CA72D83122F112F08831687008312D1
:101B600007158316A1017208A000A100A001710849
:101B7000A0070318A10A210CF600200CF500F60CB2
:101B8000F50CF60CF50CF60CF50CF60CF50CF60C49
:101B9000F50C0330F6058312A7018B1BA7178B13D7
:101BA000760803179A00750899008A1103134420D8
:101BB0008A15A71B8B173F088316C70083123E08A0
:101BC0008316C60083123D088316C50083123C08A5
:101BD0008316C4007A08CB007908CA007808C900C7
:101BE0007708C80083120020831037088316C300CB
:101BF000831236088316C200831235088316C1008B
:101C0000831234088316C0007A08C7007908C6001A
:101C10007808C5007708C4008A1183126D238A15DD
:101C200077088316A0007808A1007908A2007A0836
:101C3000A3008312A7018B1BA7178B13740803172C
:101C40009A00730899008A11031344208A15A71B70
:101C50008B1783162308C7002208C6002108C50079
:101C60002008C4007A08CB007908CA007808C900A7
:101C70007708C80083120020831033088316C3003E
:101C8000831232088316C200831231088316C10002
:101C9000831230088316C0007A08C7007908C6008E
:101CA0007808C5007708C4008A1183126D238A154D
:101CB00077088316A0007808A1007908A2007A08A6
:101CC000A3008312A7018B1BA7178B13760803179A
:101CD0009A00750899008A11031344208A15A71BDE
:101CE0008B173B088316C70083123A088316C60079
:101CF000831239088316C500831238088316C4007E
:101D00007A08CB007908CA007808C9007708C800AB
:101D100083120020831083162308C3002208C20008
:101D20002108C1002008C0007A08C7007908C60051
:101D30007808C5007708C4008A1183126D238A15BC
:101D40007A08FE007908FD007808FC007708FB009F
:101D50007E088316C7007D08C6007C08C5007B0886
:101D6000C4008830CB002030CA000230C9007B306C
:101D7000C8008312002077088316A0007808A1000D
:101D80007908A2007A08A30083102308C300220860
:101D9000C2002108C1002008C000C701C6014830A8
:101DA000C5008430C4008A1183126D238A158A11FC
:101DB0000A16062D470884008313481883178316D4
:101DC00028088000840A80018312C70A0319C80A00
:101DD000080080080319002FF2010408F1007210B6
:101DE000831B721400088316A8008312DA26710878
:101DF0008400831372188317840A0319850AE92E55
:101E00008A110A16652D8316A6010408A50026105E
:101E1000831B2614720EF038A100A107E23EA20037
:101E2000323EA40072080F39A207A207A407E93EB8
:101E3000A300A307A307710E0F39A307A407A30DDF
:101E4000A40DA409A40D71080F39A407A10D073032
:101E5000A0000A30A407A303031C2A2FA307A20390
:101E6000031C2E2FA207A103031C322FA107A003DE
:101E7000031C362FA030840083130730250525135B
:101E80008407A4300402031925170008F700031D76
:101E9000512F251B512F251A652FA519512F2030A1
:101EA000542FA51525123030F707F2010408F10070
:101EB0007210831B72147708A8008312DA26710847
:101EC00084008313721883178316840A251F412FF9
:101ED00083128A110A169A2DF701F801F901FA0105
:101EE0008316B001B101B201B3012F082E042D04F5
:101EF0002C040319AB2F2030B4000310A80DA90D3A
:101F0000AA0DAB0DB00DB10DB20DB30D2F083302FC
:101F1000031D942F2E083202031D942F2D08310229
:101F2000031D942F2C083002031CA52F2C08B0028F
:101F30002D08031C2D0FB1022E08031C2E0FB20218
:101F40002F08031C2F0FB3020314F70DF80DF90D22
:101F5000FA0DB40B7D2FB030840083138312080078
:101F6000F21BC42F0F30F700710EF7050A3077020D
:101F70000318BD2F3030F707BF2F7208F707770817
:101F80008316A8008312DA260F30F1050A30710299
:101F90000318CC2F3030CE2FF2137208F1077108DE
:0E1FA0008316A8008312DA268A110A168A2FE9
:1020000004088316A0007508A20003192628740886
:10201000C7007308C6007208C5007108C400CB0170
:10202000CA012030C9008230C8000A128A15831202
:1020300000200A168A117A08F4007908F30078085B
:10204000F2007708F1008316A20B07287408AB0092
:102050007308AA007208A9007108A8002808B63CF5
:10206000A800FA012908AC00A9170310A90CAA0CB2
:10207000AB0CFA0CF90CF80CF70CA80B3528AC1FBC
:102080004C28F709F809F909FA09F70A0319F80AB7
:102090000319F90A0319FA0A7A08F4007908F30017
:1020A0007808F2007708F100F41F6328A003A01657
:1020B000F109F209F309F409F10A0319F20A031903
:1020C000F30A0319F40A3B30A7009A30A600CA307D
:1020D000A500A4010A30A20075080319A00A74081B
:1020E000AB007308AA007208A9007108A8002708AD
:1020F000AF002608AE002508AD002408AC000A1287
:102100008A1583126C270A168A110008F100840AC6
:102110000008F200840A0008F300840A0008F400B2
:10212000FD308407F708031DAC28750A83162202C8
:10213000031D9C288312AC2820080319AF280F39EF
:1021400022020319A5280318F728A01BF728201B33
:10215000AF282030ED28831220308316A005A01E62
:10216000C328A0127508031DA0037708A0002D3016
:10217000A8000A128A158312DA260A168A11831613
:102180002008F700A00175082202031DD728770850
:10219000A0002E30A8000A128A158312DA260A1629
:1021A0008A1183162008F7002030A0050030303057
:1021B000A01EED28A0127508031DA0037708A0003B
:1021C0002D30A8000A128A158312DA260A168A11FF
:1021D00083162008F700A0013030F7077708A80021
:1021E0000A128A158312DA260A168A11831627081C
:1021F000AB002608AA002508A9002408A800AF0102
:10220000AE01AD010A30AC000A128A1583126C27A8
:102210000A168A117A088316A7007908A60078089A
:10222000A5007708A400A20B6F2883120800840180
:1022300083131F308305713083168F000F08031737
:1022400087110C3003139900A2309800903083124C
:102250009800C101C001C501C401C301C2018316B8
:1022600003170908C039890003131F129F12003099
:102270000317880083128701880189010313A801CD
:10228000A901AA013030AB002E30AC003130AD00D6
:10229000AE01FF30AF00C701C801CA01C9017130EA
:1022A00083168F000F0809308312031785000F3043
:1022B000F700031381018130840083130008F03993
:1022C0000738800064000008F739F719F0397704FF
:1022D00080006400831603170908C03989000313BE
:1022E0001F129F12003003178800831203131F135D
:1022F0009F1383169F1783121F1483160108C73973
:10230000283881000F30831290000030F8009200CE
:1023100000308316920083122F152F088316870032
:102320008312970183169B019C0101309D0083124B
:10233000031787018801890103139412AF122F0834
:102340008316870083122F162F08831687008312A7
:10235000AF112F088316870022308312940040307B
:102360008316940083122F112F088316870083127F
:1023700007150A12602A0A1683160C1483128B168C
:10238000C0308B0464000A12442B0A160A12B32CC4
:102390000A164610781846140A120B2F0A16640003
:1023A000D401D801D701D601D501DC01DB01DA0166
:1023B000D901E001DF01DE01DD01E401E301E20119
:1023C000E1010430F100FA308316AF000A128312E3
:1023D00030230A16F10BE3290A128A1577280A1608
:1023E0008A117708F1007808F2007908F3007A087A
:1023F000F400F6010408F5007610831B76148310B0
:1024000074088316C3007308C2007208C100710803
:10241000C000C7016630C6005530C5008D30C4000D
:102420000A1283126D230A16750884008313761826
:1024300083177A08E8007908E7007808E60077084B
:10244000E500F201F101DC01DB01DA01D9010A1238
:1024500007230A1603308316AB000A128312BA2729
:102460000A16831628107818281428184B2A0A12DE
:102470008A1583124E210A168A110A128A157721AB
:102480000A168A1179088316AA007808A900290873
:10249000F8002A08F9007908F2007808F1000A1219
:1024A000831207230A1605308316AB000A12831223
:1024B000BA270A1683162810781828142818742AA0
:1024C0000A128A1583124E210A168A110A128A15D7
:1024D00077210A168A1179088316AA007808A900BC
:1024E0002908F8002A08F9007908F4007808F300B0
:1024F0007208A9007108A8007408AB007308AA004C
:102500008312A7018B1BA7178B138316290883122D
:1025100003179A00831603132808831203179900E0
:102520000A12031344200A16A71B8B177708831679
:10253000B0007808B1007908B2007A08B300C7008B
:102540003208C6003108C5003008C4000A30CB008C
:10255000D730CA002330C9007830C8000A128A1563
:10256000831200200A168A1177088316B0007808B3
:10257000B1007908B2007A08B30083143308C300AD
:102580003208C2003108C1003008C000C701C601CE
:102590002030C5008430C4000A1283126D230A164D
:1025A0007A08D8007908D7007808D6007708D500CF
:1025B000A7018B1BA7178B1383162B0883120317F6
:1025C0009A00831603132A088312031799000A122C
:1025D000031344200A16A71B8B177A088316AF0033
:1025E0007908AE007808AD007708AC002F08C70066
:1025F0002E08C6002D08C5002C08C400BD30CB0035
:102600005230CA001630C9007A30C8000A128A1542
:10261000831200200A168A118310C5308316C30066
:10262000FE30C2008230C1008030C0007A08C7008E
:102630007908C6007808C5007708C4000A1283121A
:102640006D230A1677088316B0007808B100790860
:10265000B2007A08B3002F08C7002E08C6002D0864
:10266000C5002C08C4002F08CB002E08CA002D0876
:10267000C9002C08C8000A128A15831200200A1605
:102680008A1177088316B4007808B5007908B60077
:102690007A08B700C7003608C6003508C5003408F8
:1026A000C400F630CB002430CA00D630C9006B30ED
:1026B000C8000A128A15831200200A168A11831094
:1026C00083163308C3003208C2003108C100300845
:1026D000C0007A08C7007908C6007808C5007708E6
:1026E000C4000A1283126D230A167A08FE007908C4
:1026F000FD007808FC007708FB0083145808831657
:10270000C300831257088316C2008312560883162B
:10271000C100831255088316C000C701C6014830A6
:10272000C5008330C4000A1283126D230A1677088D
:102730008316B0007808B1007908B2007A08B300B7
:10274000AC30C700C530C6002730C5007130C400AA
:102750002F08CB002E08CA002D08C9002C08C8007D
:102760000A128A15831200200A168A1183100A3071
:102770008316C300D730C2002330C1007830C000B8
:102780007A08C7007908C6007808C5007708C40031
:102790000A1283126D230A1683163308C700320803
:1027A000C6003108C5003008C4007A08CB0079089B
:1027B000CA007808C9007708C8000A128A1583126F
:1027C00000200A168A1177088316B0007808B10035
:1027D0007908B2007A08B30083103308C3003208C6
:1027E000C2003108C1003008C0007E08C7007D0863
:1027F000C6007C08C5007B08C4000A1283126D2342
:102800000A167A08DC007908DB007808DA00770815
:10281000D9008316BF01BE014630BD008530BC0023
:1028200083125C088316C30083125B088316C20000
:1028300083125A088316C100831259088316C000F8
:102840000A128A158312E2210A168A11031C2E2C01
:10285000DC01DB014830DA008530D9005C088316E2
:10286000BF0083125B088316BE0083125A088316CA
:10287000BD00831259088316BC00CD30C300CC3094
:10288000C2004C30C1007B30C0000A128A1583128E
:10289000E2210A168A11031C552CCD30DC00CC3005
:1028A000DB004C30DA007B30D900831058088316E7
:1028B000C300831257088316C2008312560883167A
:1028C000C100831255088316C0003330C70093300F
:1028D000C6000830C5008730C4000A1283126D2379
:1028E0000A167708F1007808F2007908F3007A08F0
:1028F000F4008316C7007308C6007208C50071088B
:10290000C400CB01CA014830C9008530C8000A1292
:102910008A15831200200A168A117A08D8007908CD
:10292000D7007808D6007708D5000A128A15682AD9
:102930000A168A117A08E0007908DF007808DE00BC
:102940007708DD000A128A155A2B0A168A117A08AE
:10295000E4007908E3007808E2007708E100461C0B
:102960002D2D0A128A15352C0A168A117708F100C6
:102970007808F2007908F3007A08F400F6010408F8
:10298000F5007610831B7614831074088316C30039
:102990007308C2007208C1007108C0003330C7005C
:1029A0009330C6000830C5008730C4000A12831275
:1029B0006D230A1675088400831376188317770829
:1029C000F1007808F2007908F3007A08F400831621
:1029D000C7007308C6007208C5007108C400CB01A7
:1029E000CA014830C9008530C8000A128A1583120E
:1029F00000200A168A117A08EC007908EB007808A2
:102A0000EA007708E9000A128A15112D0A168A11C0
:102A10007708F1007808F2007908F3007A08F400EA
:102A20008316C7007308C6007208C5007108C40089
:102A3000CB01CA012030C9008230C8000A128A15B1
:102A4000831200200A168A117A08F0007908EF0034
:102A50007808EE007708ED00352DEC01EB01EA0176
:102A6000E901F001EF01EE01ED012130F700F70B74
:102A7000372D24300C1E3A2D99002130F700F70B2A
:102A80003F2DC8014B30C70041308316A8000A1201
:102A90008A158312DA260A168A1157308316A8007F
:102AA0000A128A158312DA260A168A1153308316FF
:102AB000A8000A128A158312DA260A168A112B3008
:102AC000840083130A128A15E92E0A168A1120300F
:102AD0008316A8000A128A158312DA260A168A11AA
:102AE000D3014B30530784008313800803198E2DC4
:102AF0002130F700F70B7A2D4B30530784008313F6
:102B00000008F10071080C1E832D99005308D30AA8
:102B10004B3E840083130008D406712DC8014B304E
:102B2000C700103084004A08F2004908F1000A1278
:102B30008A15032F0A168A1120308316A8000A125C
:102B40008A158312DA260A168A11D3014B305307ED
:102B50008400831380080319C32D2130F700F70B7D
:102B6000AF2D4B305307840083130008F100710828
:102B70000C1EB82D99005308D30A4B3E84008313D2
:102B80000008D406A62DC8014B30C70004308400CD
:102B90006808F4006708F3006608F2006508F100B1
:102BA000F501002020308316A8000A128A1583122E
:102BB000DA260A168A11D3014B3053078400831397
:102BC00080080319F92D2130F700F70BE52D4B3064
:102BD0005307840083130008F10071080C1EEE2DCA
:102BE00099005308D30A4B3E840083130008D4068F
:102BF000DC2DC8014B30C700043084005808F400B5
:102C00005708F3005608F2005508F100F5010020BE
:102C100020308316A8000A128A158312DA260A16B3
:102C20008A11D3014B3053078400831380080319A2
:102C30002F2E2130F700F70B1B2E4B30530784004B
:102C400083130008F10071080C1E242E990053080C
:102C5000D30A4B3E840083130008D406122EC80109
:102C60004B30C700023084005C08F4005B08F300BE
:102C70005A08F2005908F1000130F5000020203018
:102C80008316A8000A128A158312DA260A168A11F8
:102C9000D3014B3053078400831380080319662E39
:102CA0002130F700F70B522E4B305307840083136B
:102CB0000008F10071080C1E5B2E99005308D30A1E
:102CC0004B3E840083130008D406492EC8014B30C4
:102CD000C700043084006008F4005F08F3005E0859
:102CE000F2005D08F100F501002020308316A800F5
:102CF0000A128A158312DA260A168A11D3014B307A
:102D0000530784008313800803199C2E2130F70099
:102D1000F70B882E4B305307840083130008F10013
:102D200071080C1E912E99005308D30A4B3E840063
:102D300083130008D4067F2EC8014B30C700023031
:102D400084006408F4006308F3006208F20061087C
:102D5000F1000130F500002020308316A8000A128F
:102D60008A158312DA260A168A11D3014B305307CB
:102D70008400831380080319D32E2130F700F70B4A
:102D8000BF2E4B305307840083130008F1007108F5
:102D90000C1EC82E99005308D30A4B3E840083139F
:102DA0000008D406B62EC8014B30C700043084009A
:102DB0006C08F4006B08F3006A08F2006908F1007F
:102DC000F501002020308316A8000A128A1583120C
:102DD000DA260A168A11D3014B3053078400831375
:102DE00080080319092F2130F700F70BF52E4B301F
:102DF0005307840083130008F10071080C1EFE2E97
:102E000099005308D30A4B3E840083130008D4066C
:102E1000EC2EC8014B30C700043084007008F40069
:102E20006F08F3006E08F2006D08F1000130F50044
:102E3000002020308316A8000A128A158312DA2691
:102E40000A168A11D3014B3053078400831380087C
:102E50000319402F2130F700F70B2C2F4B3053076D
:102E6000840083130008F10071080C1E352F9900AF
:102E70005308D30A4B3E840083130008D406232F43
:102E8000C8014B30C700023084004508F4004408F4
:102E9000F3004308F2004208F1000130F500002081
:102EA00020308316A8000A128A158312DA260A1621
:102EB0008A11D3014B305307840083138008031910
:102EC000772F2130F700F70B632F4B305307840027
:102ED00083130008F10071080C1E6C2F9900530831
:102EE000D30A4B3E840083130008D4065A2FC8012E
:102EF0004B30C7002A308316A8000A128A158312A5
:102F0000DA260A168A115408F1003730F2000A1244
:102F10008A15B02F0A168A110D308316A8000A12DE
:102F20008A158312DA260A168A110A308316A80037
:102F30000A128A158312DA260A168A11D3014B3037
:102F400053078400831380080319B62F2130F7003C
:102F5000F70BA82F5308D30A4B3E840083130008B5
:102F6000F10071080C1EB22F99009F2F2130F7003D
:102F7000F70BB82F6400C90A0319CA0AD0296300E5
:0639C0008A010028080046
:1000080000000000000000000000000000000000E8
:080018000000000000000000E0
:04400E00FD2CFF3F47
:00000001FF
